:030000000208AA49
:080003000280038E828F83222C
:08000B0002800BAE82AF8322DC
:08001300028013742D0173003B
:08001B0002801B11730171004A
:08002300028023111601710097
:03002B0002802B25
:10002E00217601730167216521872194018A01CE12
:10003E0021CE21A802092A020A85017D0201BB02F6
:10004E0009CE0209D4020A1202086B020831020715
:10005E00BC02079202094D214A3098FDC298E599DB
:10006E0022117174203099FDC299F59922117DC02B
:10007E00E0740D1173740A1173D0E022C2D51162AF
:10008E0031A8B41B03D3E422B40D05D2D5C3E422A8
:10009E00FA314A40E9CA1173116231A8B41B0280C9
:1000AE00E4B40D03EAC322B40804117380D0B4156E
:1000BE000280F7FB314A40E0CB1173EAC44BC322F6
:1000CE007A007B007C04C2D5116231A8B41B07D321
:1000DE00E4F583F58222B408028003B47F0CBC04DD
:1000EE000280E5117331390C80DEB40D108B838ADA
:1000FE0082BC0407E4F583F582D2D5C322FD314AD2
:10010E0040C6CD120073EDC0E03128D0E02AFAE4EB
:10011E003BFBDCB4C38A828B8322EBC454F0FBEA34
:10012E00C4540F4BFBEAC454F0FA22EAC4540FFA3B
:10013E00EBC454F04AFAEBC4540FFB22C324D05044
:10014E001424F64004240AC32224F9500824FA4049
:10015E00042410C322D322C0E0C4540F24F650024C
:10016E002407243A1173D0E0C0E0540F24F6500255
:10017E002407243A1173D0E022C0E0E5833165E50F
:10018E00823165D0E022C0E0E493A3600AA2E75476
:10019E007F1173400280F1D0E022C0E0C394614031
:1001AE0009941A5005D0E024E022D0E0227800C055
:1001BE00E0E4936008A2E7084003A380F4D0E022B5
:1001CE00C0E0C3309808E599B41B01D3C298D0E0C3
:1001DE0022900D213194EF3165EE3165319411622B
:1001EE0031A875F0DFC0F075F001C0F0F5F0901099
:1001FE0000F1925024758204E493B4FE150582E456
:10020E0093B5F00E11717582203194117D75824077
:10021E00E4730583E583B400D8E5F0B43F07900E90
:10022E00871145A1D6B44D07900E8F114581C6B4E6
:10023E005207900E941145A13DB44C07900ECE314D
:10024E009441A8B45507900E9B1145C14BB44E076F
:10025E00900E9E1145E13DB44A07900EA2114581C4
:10026E0014B44807900EA81145814BB44507900E63
:10027E00B41145818CB44307900EB91145E119B400
:10028E005A0B74006012900EBD1145E14DB4490831
:10029E00900EAE1145020773017D900DB911457890
:1002AE00107A10760008DAFB1167B41B028074B462
:1002BE003A0679007143800A314A40EC790671435F
:1002CE0080E67C007162F87162F5837162F582716D
:1002DE0062B40104D29780317026E860187162FA18
:1002EE0079017143EAA2E7929712086BE43402F99E
:1002FE007143A3D8E57162EC60AE7904714380A8B6
:10030E00E860F27162D8FC80ECE860047162D8F3A8
:10031E007162EC70E5713A900DD8114530987A11F2
:10032E00678076713A900DD01145806D7800790016
:10033E00D9FED8FA22E95407232410F907E77002F0
:10034E00090722D3878209878309E5827005E58331
:10035E007001C322116731A8B41B06D0E0D0E08033
:10036E00C2B43A0A79057143D0E0D0E041D0314AA7
:10037E0050067907714380DCFA116731A8B41B026D
:10038E0080D9B43A0280DD314A5006790771438034
:10039E00E8CAC44AFA2CFCEA22EEC0E0EFC0E090B4
:1003AE000DDF114579107EE87F0D91107EEE7F0DE9
:1003BE0091107EF37F0D91107A0571514009DAFA92
:1003CE00900E2F11458025900DFE114579167E0257
:1003DE007F0E91027E137F0E91027E1B7F0E910285
:1003EE007E217F0E91027E267F0E9102D0E0FFD0FD
:1003FE00E0FE017D715150091171120A12110611A0
:10040E004522715180F2900D601145110631879091
:10041E000D2E114511CE20D5065002E114110E11EC
:10042E007D900E3D11451106E4F5D0F5F0F8F9FA80
:10043E00FBFCFDFEFF758108C0E0C0E0737A101171
:10044E007B11063187743A111E7B101106E493A3BB
:10045E0031651171DBF7116F7B101106E493A35414
:10046E007FB47F01E424E04001E424201173DBEC2F
:10047E00117DD1D0110E31CE4002DAC5017D900D25
:10048E00A2114511CE110E117D3187743A111E74D1
:10049E00281173110EE4933165900D7B1145118A6D
:1004AE0020D510400E110612086B117D1106A311F6
:1004BE000E8197900DAE0145900D6A11457815117C
:1004CE0071D8FC1145758310F1924002017D116FB8
:1004DE00758220319475822031BB7421C398F874D3
:1004EE00201173D8FC758200318778067420117341
:1004FE00D8FC758204E493AA83B4FE05900E758031
:10050E0018B4FD05900E7C8010B42305900E7980F2
:10051E0008B4F90280EE900E8311458A83117D7422
:10052E00FFB5830281DA0583E583B4009B81DA117E
:10053E007B7AFF90100015830583E583B40002805B
:10054E0021F192501D758204E4934403F460E91185
:10055E006F0A74412A111E11267582203194117D65
:10056E00A146BAFF05900D370145900D291145742E
:10057E00411173111674412A1173900D2E114511EC
:10058E0062B41B02017DFB741FC39AEB400231A8BB
:10059E001173FB117DEBC3944140CFFBEAC39B402B
:1005AE00C90B90100015830583E583B400028017F4
:1005BE00F1925013758204E4934403F460E9DBE78F
:1005CE00117D758240813622900E5D11457C3F90E3
:1005DE000E8AD1407C4DD1407C52D1407C4CD140D2
:1005EE007C55D1407C4ED1407C4AD1407C48D14094
:1005FE007C49D1407C45D1407C43D140740060049D
:10060E007C5AD140900E6B1145901000F192502003
:10061E00758204E493B4FE11116F0582E493117395
:10062E0011267582203194117D0583E583B400DC9B
:10063E00017D116FEC117311261145017DD1E290F0
:10064E000E471145EB3165EA31651145ED3165EC2B
:10065E003165117D8D838C82A3AC82AD83900D5656
:10066E0011451167B41B02E112117D8A828B83EC56
:10067E00C39582FAED95837009EA603254F07002E8
:10068E0080027A10743A1173EA31653187E5832559
:10069E00822AFBE43165E49331652BFBA3DAF7EB99
:1006AE00F4043165117DD1D031CE50C38056743AE9
:1006BE001173E431653165316504316574FF31655F
:1006CE00017BE8C0E0780CE58C04000070FBD8F7E5
:1006DE00D0E0F822117B900D84114511CE402120DF
:1006EE00D51EC083C082117D900D8E114511CEADE9
:1006FE0083AC82D0E0FAD0E0FB400520D502017D2C
:10070E00D0E0D0E0117D900D190145D1E2900D9809
:10071E001145116231A8B459EB117B8B838A82E4A7
:10072E0012086BEDB58305ECB5820122A380F09023
:10073E000D4D114511CE40CE20D5CB110E017B11A2
:10074E007B900EBD1145742C111E900D9811451104
:10075E006231A8B459AE117B1207BC900EC2500381
:10076E00900EC90145117D7800117DE83165743A0E
:10077E0011731171E6316508E8540F70F5117DB8EB
:10078E0000E9017D758200E493B4A517A3E493B448
:10079E00E511A3E493B4E00BA3E493B4A50575822D
:1007AE0000D32274FFB58302C322058380D6740062
:1007BE006038908000E493F4700DA37400B582F558
:1007CE007400B583F0C322908000E4936006E412B7
:1007DE0008314016A37400B582F07400B583EB9017
:1007EE0080007CE87D04DC04DD02D3227420A2AFFD
:1007FE0092D1C2AFF0F07B147AE5DAFEDBFA74A088
:10080E00F07A05DAFEE493A2D192AFF470D8A37415
:10081E0000B583EA7400B582E574FF908000F0E4C1
:10082E00F0C322F5F0EAC0E0EBC0E07A197440A202
:10083E00AF92D1C2AFF0E5F0F07B13DBFE74C0F0E7
:10084E007B05DBFEE493A2D192AFC395F06003DA91
:10085E00DCD3E4F0D0E0FBD0E0FAE5F022C0E0C05B
:10086E00F0F5F07400601BE583B4FF02800B5012AC
:10087E00B48002800450028009E5F01131D0F0D02E
:10088E00E022E5F0F0E493C395F06009E0C395F043
:10089E006003D38001C3D0F0D0E02232E4F5A8F596
:1008AE00B875D00011A911A9F4F580F590F5A0F551
:1008BE00B075813079C87AF9DAFED9FA740060130E
:1008CE0074B5600F78FAA2B579C8D9FE4005D8F68E
:1008DE001207BC75F0F911FD312A75F0FD11FD906E
:1008EE000EE212019412007D7E007F800201DF90E5
:1008FE0010001207925024758204E493B5F015C0CF
:10090E00F0C083741EC0E07409C0E0758240E473C9
:10091E00D083D0F00583E583B400D72274FAF57B3B
:10092E00F57AF579F578637A556379CC63781DF5A8
:10093E008DF58B758921758780759852D28E2230F0
:10094E009806120067B41B51120067B41B4B31BBE3
:10095E00209803741B22120067B45B4431BB30989D
:10096E00DE120067B44103740B22B44203740A22F0
:10097E00B44303741522B44403740822B4350280C0
:10098E0007B4360280028018C0E031BB30980B12DB
:10099E000067B47E09D0E024E422D0E080A1D0E04C
:1009AE0031BB30989A120067B41BF580A1EAC0E003
:1009BE007A14E58C2098050470FADAF6D0E0FA2263
:1009CE00C0F0C0E08013C0F0C0E030E70C742D1210
:1009DE000073D0E0C0E0F4240175F06484D2D560D9
:1009EE0007C2D52430120073E5F075F00A8430D5B5
:1009FE000260052430120073E5F02430120073D02B
:100A0E00E0D0F022C0E0E8C0E0C2D5AA82AB837C81
:100A1E00107D27517060072430120073D2D57CE808
:100A2E007D035170700330D5072430120073D2D578
:100A3E007C647D005170700330D507243012007332
:100A4E00D2D5EAABF075F00A84700330D5052430A8
:100A5E00120073E5F08BF02430120073D0E0F8D062
:100A6E00E022780008C3EA9CFAEB9DFB50F618EAE8
:100A7E002CFAEB3DFBE822C0E0E8C0E0E9C0E0EC78
:100A8E00C0E0D2D1D2D5E493A3602520E72E547FC7
:100A9E00B40D0712007DD2D180ECB41F04C2D580F4
:100AAE00E5B40E0512007D8007C2D112007380D608
:100ABE00D0E0FCD0E0F9D0E0F8D0E022547FF8206E
:100ACE00D103120071C2D1C082C083900B3F7C0053
:100ADE00E86007F9712E70FCD9FA712E603CB40FE4
:100AEE0012712E0483801E68667767796278766B42
:100AFE00716A7A0483800E657461726E69736F6CAD
:100B0E00756D706463A2D592E5D2D5B81402C2E5B4
:100B1E00B80C02C2E512007380C0D083D08241941B
:100B2E00E493BC00057CFF540F227C00A3C4540F39
:100B3E00228290E82386054CF844B3B0B1485FF0AA
:100B4E00117FA0157F1C2ED1405A50F103BFBA0C55
:100B5E002F96018D3F95380D6F5F1207710E562F30
:100B6E00483B6258201F7670322440B840E1618FB6
:100B7E0001340BCA89D3C0A3B9588004F80285602A
:100B8E002591F092731F107F12549310444807D191
:100B9E0026564FD0F66472E0B83BD5F0164F56305D
:100BAE006F48025FA8201F017630D5602541A42C26
:100BBE0060056F013F261F30078E1DF06399F042CE
:100BCE00B8201F2330027AD1602FF0F6058F931ACA
:100BDE005028F082046FA30D3F1F514023013E05A4
:100BEE0043017A01176493302A088C243099B0F3AC
:100BFE001960254135098ECB191230051F311D04A0
:100C0E00144F761204AB279056012FA8D5F0AA26C2
:100C1E00205F1CF0F361FE0141730127C1C0848F78
:100C2E00D6018770564F19701FA8D99076021743B8
:100C3E00FE01C1840B157F028B14308F63396F193F
:100C4E00F011C9106D023F91097A41D0BA0C1D39CD
:100C5E005F07F2111720416B3509F775120BA7CC00
:100C6E0048023F6412A00C27E39FC0147770114016
:100C7E007121C0682541F0627FD1D021E16258B068
:100C8E00F3051F733077B16F19E01943E0582FF653
:100C9E00A414D02303FE31F5143099F8033F6422D7
:100CAE00516025412FE30156279309FE11FE79BAB3
:100CBE00607542EA6258A0E51F534FD1C0A30942A6
:100CCE0053F71204621B30F505F7690C351B708261
:100CDE002F2F144F51C064250057656C636F6D65DF
:100CEE008094322C2062791FF81FFE0D0E202053A7
:100CFE00656594322E444F432C94322E455155A4A3
:100D0E0094322E484452B4D58D2E0E201F9E1FA015
:100D1E00210D0E414444523A003EA086CA8228005C
:100D2E00292C958C80C83A20001F9782C373C7A6C2
:100D3E00832CBA204A554D508086A172820D0E0D1D
:100D4E000D1F8783813A20001FE4FB206B65793AE3
:100D5E0020000D0D1F888083812028000D0D1F821D
:100D6E001FFD001F8120202020201FC90E29201FBB
:100D7E00871FB23A200046697273741F813A2000B1
:100D8E004C6173741F813A2020001FB9A120737526
:100D9E0072653F000D0D416464726573733E2000F1
:100DAE0020201F9CC12C8E81F70D0E0D0D1F9F2034
:100DBE006173636969F9961F9884892C958C80A05C
:100DCE000D0E0D1F8AA065640D0E0D1F8AC1640DD8
:100DDE000E53756D6D6172793A0E20C67391640E65
:100DEE00208B91640E208B207772697474656E0E61
:100DFE001F9B3A0E208B20756E61626C658020778A
:100E0E00726974650E2020626164F5730E20859FF1
:100E1E0096C60E2085849D0E2085206E6F6E849D55
:100E2E000E1F979B2064657465637465640D0E0DCB
:100E3E00866E696E67823A0D0E0D0D53656E64698E
:100E4E006E671F988489AC20200020802020000D22
:100E5E000D5374616E646172641F9E730E1FDA1FF0
:100E6E00F465641F9E730E1F9A9E001F82001F8FD3
:100E7E001FE21FAA003F3F3F001FD7001F8ED7D192
:100E8E00001FD18273001F8682001F8A001F9300ED
:100E9E001F8781001F88808381001F84DB9A830057
:100EAE001F84DBC083001F9C9A92001FED83001FDE
:100EBE00CB9990001F9990CB640D0E1F859B0D0E44
:100ECE004C6F616420496E74656C2068657820668D
:100EDE00696C65000D0A0A38303531534243204D96
:100EEE006963726F70726F636573736F72204C6596
:0F0EFE0061726E696E6720426F6172640D0A0047
:10100000A5E5E0A5FE44000000000000000000008F
:10101000000000000000000000000000FFFFFFFFD4
:0F102000446973617373656D626C65000200480B
:10104000112C7D14C2D1114CDDFC012CEFF5835124
:101050004FEEF582514FE493FAA3E493FBA3E4939C
:10106000FCEA5408700FEA035478F8EA54074890F1
:1010700016C8938008EAC4540F901362935403F87F
:101080002EFEEF3400FF743A512A719D20D121EADF
:10109000514F719DB80104790B8011EB514F719D37
:1010A000B8020479088005EC514F7906719DD9FC8E
:1010B000EA54087010901748EA035478F8EA540785
:1010C0004893F980099017C8EAC4540F93F9901E09
:1010D000947808C374204007E99309A2E7547F512C
:1010E0002AD8F1741BC0E07411C0E0EA5408700FF4
:1010F000EA035478F8EA5407489016C8938008EA3F
:10110000C4540F9013629354FC03031490111D23D5
:101110002582F582E43583F583E473012C412D416A
:101120003C21812172414841044152415821A22170
:10113000D7415E4169416D4108411021AA218321B7
:101140007441714177417D413E411C418121DF4124
:101150001441C54185418B41914195419B41A94134
:10116000AF41B541BB410C41BF41CB41D741E74104
:10117000ED2231F67440512A7452512AEA54014149
:101180004531F6EB20E703EB414F9012F5E493A3D2
:1011900060F5F8C39B7003020038E493A330E7FACC
:1011A00080EB511031F8742F512AEB547823C4F896
:1011B000EB54806014901372E893901F293582F5E8
:1011C000825002058331978005E82420514F742E08
:1011D000512AEB5407414531F6318331F8ECFBEBF2
:1011E0002EF582EB20E703E48002E4F43FF583026E
:1011F00000367440412A5108742C512A7420412A27
:101200007423412A318331F87441412A31AA31F8DB
:101210007443412A31F25108742B512A7444512AE3
:101220007450512A7454512A7452020030EF54F809
:10123000F8EAC403540748514FEB414F31F674525A
:10124000512AEA540702002E510831F85100EB02EE
:1012500000343183ECFB414A511031F821AA510886
:1012600031F85100EB514F21DB513E416031744167
:101270006051087442412A513E31F821DF31832107
:10128000DB31AA21DB513E31F84108513E31F821D2
:1012900083513E414A318331F8413EEBC0E0ECFBE3
:1012A000318331F8D0E0FB2183318331F82174316F
:1012B0007431F84108317431F821833174414A5155
:1012C0001C31F85100EB514FEC414F31F631F251E6
:1012D00008742B512A411C31F631F25108742B51FC
:1012E0002A7450512A411031F631F2411C31F25129
:1012F0001C31F84108E04143C38153D0824450CCB3
:10130000834450C88050B09050B1A050B2B050B398
:1013100099534255C6CD5448B2C85432434FCECCEF
:10132000544CB2CB5243415032C8CA52434150325E
:10133000CC8C5448B08A544CB08D5448B18B544C2A
:10134000B1F0C2D05053D7A849C5B849D089544D3F
:101350004FC48854434FCE9853434FCE8750434F8A
:10136000CE00595909090909097A7E0976330952CB
:101370000971000206080C0E101214161B1E202301
:101380002425F8F0E493C398227950E58DF404F80D
:10139000D8FED9F722514F743A412A514F74204157
:0113A0002A22
:10140000A5E5E0A5FE53000000000000000000007C
:10141000000000000000000000000000FFFFFFFFD0
:0C14200053696E676C652D537465700095
:1014400030B306901D1B020045900013E49324FE68
:101450006005901D3E8146A393F8E4A393F582882E
:101460008374027182700EA3741471827007A37466
:10147000EF71826011A882A983901D4B9146E951BA
:101480004FE8514F012CE5B85404F5B8901CFE917B
:1014900046EF514FEE514F901CE8914612003C2010
:1014A000D50D5007901D073197012CAE82AF83C236
:1014B0008A901D5A9146901E523197E4758108C05A
:1014C000E0C0E08E828F83F5D0F8F9FAFBFCFDFED8
:1014D000FFF5F0757CDD757D14D2AAD2AF737189EA
:1014E000D0E0F9D0E0F8D082D083D0D0D0E032C0C4
:1014F000E0C0D0C083C082E8C0E0E9C0E07189D21A
:1015000099719D719DE58124FBF8E6719BE5F07171
:101510009B08E62354015145719D08E6514F08E6AA
:10152000719B719D08E6719508E67195EA7195EBDE
:101530007195EC7195ED7195EE7195EF719B719DC3
:10154000E824F8719B719D719DE57C8E7CFEE57DA4
:101550008F7DFFEAC0E0EBC0E0ECC0E0D2D1114CDF
:10156000D0E0FCD0E0FBD0E0FAAF7DAE7CE581249A
:10157000F9F8E6F57C08E6F57D120062120040B449
:101580000D0281DEB4200281DEB43F07901DCB91B5
:1015900046A179B45113901E4B3197C2AA71897537
:1015A000080075090075810932B44802A1CDB45212
:1015B00002A1FDB45302C167B44102C1AAB42E070F
:1015C000901E523197A179A179743D412A901D99BD
:1015D0003197E47195719DA88118E6719B08E651D9
:1015E0004F7802790EA1ECE871957910719DE65162
:1015F0004F08D9F8112CB800EE112CA179901344A2
:101600003197B1C9E58124FCF8E6719B901348A895
:10161000A8D16090134BA8B8D16090134EA889D17F
:1016200060901353A888D160901358A898D1609007
:10163000135DA887D1607454512A7430512AB1C9FE
:10164000E58C514FE58A514F719D7454512A743184
:10165000512AB1C9E58D514FE58B514F112CA1791C
:101660003197B1C9E8619B7817719DD8FC901D81B5
:101670003197E58124F9F8E68E7CFE08E68F7DFF40
:10168000EAC0E0EBC0E0ECC0E0D2D1114CD0E0FC0D
:10169000D0E0FBD0E0FAE58124F9F8EEAE7CF57CF1
:1016A000F608EFAF7DF57DF6A179E58124FBF89092
:1016B0001DBB319712003A400820D505F6112CA128
:1016C00079901D073197A179AD066F39394649499F
:1016D00063066F39394649496306AD39160E111153
:1016E0006306AD39160E111166061A1F160E11117A
:1016F00066061A1F160E111166061A1F160E111114
:1017000066062269161F9292660622A14D8386867E
:101710009B06969D160E11112606225D4DAD8E8EEE
:101720002606423D2F2B37374606423D390E111112
:101730004606423D39571111A5061111390E1111F6
:10174000A9068989391A89895A0E48732B2B2B2BA4
:1017500030004375212121212E0E676E06060606F4
:1017600038006A700A0A0A0A330E5D5D5D5D5D5DD0
:101770003B00121212121212410E8F8F8F8F8F8F19
:101780003E005D354C4C4C4C7C0E124F244C4C4C66
:101790004C004C4F808080805D0E4C2B57924C4CFF
:1017A00012001C1C15151515630E191984888888DC
:1017B000600078781F278B8B530E5353194C4C4C79
:1017C000530053531C4C4C4C2B21060A5D128F4C7A
:0817D0004C804C1588274C4C9D
:10180000A5E5E0A5FDFF00000000000000000000CD
:10181000000000000000000000000000FFFFFFFFCC
:0F182000454550524F4D20626F6F74696E6700DF
:0A184000900200E030E001229175F3
:10190000A5E5E0A5FE510000000000000000000079
:10191000000000000000000000000000FFFFFFFFCB
:0B192000517569636B20686F6D6500F6
:071940007E007F8002102CE5
:10195400C0D0C0E012004890197C120038D0E012C8
:10196400003412004890198B120038D0D0E5D01200
:101974000034120048020000416363756D756C61A8
:10198400746F72203D2000505357203D2000FEEB21
:10199400A4FD8EF0ECA4FCEB8EF0A4C5F02C2DC5B8
:1019A400F022E4FBFCFFE709B42D030FE709C3941D
:1019B40030B40A005012FA740A75F0001219922A0F
:1019C400FBE5F03400FC80E4EB8CF0DF002279705E
:1019D400120032B40D08770079701219A622B408E7
:1019E400061200301980E9B40C061200300980E0B8
:0719F400120030F70980D951
:101A0000A5E5E0A5FE5A000000000000000000006F
:101A1000000000000000000000000000FFFFFFFFCA
:0B1A20005A415020454550524F4D00E8
:101A4000901A6A120038743E120030120032B4311B
:101A500004718F80EBB43204712F80E4B4330491AD
:101A60007580DD7E007F8002102C0D0A32344C43DD
:101A700032353620454550524F4D2066756E6374A1
:101A8000696F6E73203120534156452C203220441B
:101A9000554D502C2033204C4F41440D0A00D2B4F8
:101AA000D2900000C2B40000C290227F083392B4EA
:101AB0009297D29000000000C290DFF1D2B4D29091
:101AC00000000000A2B4C290227F08D29000000063
:101AD00000A2B4929733C290DFF122C2B4D2900038
:101AE000000000C290D2B422C2B4D2900000000024
:101AF00000D2B422519E74A051AB40F822519E7482
:101B0000A051ABE58351ABE58251AB519E74A1511D
:101B1000AB51C951E822F5F0519E74A051ABE58359
:101B200051ABE58251ABE5F051AB51E851F4229055
:101B30001B5D12003812003C1200487A1012004857
:101B400012003674201200307B1051FDA3120034B5
:101B50007420120030DBF3DAE4120048220D0A652B
:101B60006570726F6D2061646472657373205B30A1
:101B70003030302D374646465D203E200074012629
:101B8000F608740036F622E6F58208E6F583229020
:101B90001C2312003812003C500122E582AA83C0A7
:101BA00083C0829000007116900001EA7116D08205
:101BB000D083787EE582F608E583F6901C42120019
:101BC000381219D2F4F582E5F0F4F583A312004837
:101BD000C083C082E582AA83900002711690000340
:101BE000EA7116D082D083787C7410F6087400F6FF
:101BF000C083C082787E7187E0FB787C7187EB714F
:101C000016787E717D787C717DD082D083740D12C0
:101C10000030120053A3E583458270D4901C6D12EE
:101C20000038220D0A536176652050726F67726129
:101C30006D20737461727420616464726573733EA5
:101C400020000D0A4E756D626572206F6620627904
:101C5000746573205B302D33323736385D203E207B
:101C6000000D0A536176696E672E2E2E000D446FAB
:101C70006E652E2E00901CDB12003890000051FD86
:101C8000787EF690000151FD787FF67410787CF62E
:101C9000087400F690000251FDFA90000351FDF522
:101CA000838A82C083C082787C718751FDFB787EF5
:101CB0007187EBF0787E717D787C717DD082D083E6
:101CC000A3E583458270DC90000051FDFA9000018D
:101CD00051FDF5838A82C082C083220D0A4C6F6158
:101CE00064696E672E2E2E00292C206F72203C45D1
:101CF00053433E20746F20657869743A20000D1FAD
:101D00008880838120280020436F6D6D616E642080
:101D100041626F727465642E0D0A000DA1C52063C7
:101D20006F6E6E65637420494E5431202870696E61
:101D300020313329206C6F7780BACFCC0D009432DC
:101D4000B3C7AE8120303031330D001FB8B3FFA5CB
:101D500020766563746F72AE20000D4E6F77866ECD
:101D6000696E67A6CFCC206D6F64653A20203C5227
:101D700045543E3DCC2C203F3D2048656C700D0DF8
:101D800000536B697070696E6720496E7374727569
:101D90006374696F6E2D3E20000D0A4C6F633A200C
:101DA00020496E742052414D204D656D6F7279202F
:101DB000436F6E74656E74730D0A004E6577204133
:101DC00063632056616C75653A20000D1FCF1FCCF0
:101DD0001F9E3A0D3C5245543E2086D4F60D203CC1
:101DE00053503E2086D4F60D20273F272020FF8E1B
:101DF000D70D20272E272020FFC4FD730D2027524A
:101E0000272020FF207370656369616C2066756E02
:101E10006374696F6EC4730D20274827202084DB0C
:101E2000C0920D202753272020FCD4F60D202741F7
:101E3000272020F0A2204163632076616C75650D38
:101E4000202751272020C8CFCC0D0E517569740D65
:101E50000A00202041434320422043204450545252
:101E6000202052302052312052322052332052341E
:101E70002052352052362052372020535020202027
:101E8000416464722020496E737472756374696F63
:101E90006E0D0A004143414CCC004144C400414412
:101EA00044C3414A4DD0414ECC434A4EC5434CD227
:101EB0004350CC44C14445C34449D6444A4EDA4910
:101EC0004EC34AC24A42C34AC34A4DD04A4EC24A8E
:101ED0004EC34A4EDA4ADA4C43414CCC4C4A4DD0C0
:101EE0004D4FD64D4F56C34D4F56D84D55CC4E4FF6
:101EF000D04F52CC504FD0505553C85245D4524574
:101F000054C952CC524CC352D25252C3534554C2FC
:101F1000534A4DD0535542C2535741D05843C858E5
:101F20004348C45852CC3F3FBF50B054434FCE50AB
:101F3000B153434FCE50B249C550B349D043B054CA
:0F1F400032434FCE5053D744B84143C3FDC2FE86
:20200000A5E5E0A5FE5700000000000000000000000000000000000000000000FFFFFFFF60
:0D2020004E455720434F4D4D414E44530057
:20204000758107902BBF79007AF07BD87C02EB4C601CE493A3CAC583CAC9C582C9F0A3CA76
:20206000C583CAC9C582C91BBBFFE31C80E090F2EBE4F012207690F000E0A3F5F0E0C5F0DB
:20208000C0E0C0F01227471581158112223A12279090F2E6F01225DF1220B112227F1223D4
:2020A000491223A912244312222012225002208E2290F2E6E0122AA97B61122AA0122B4470
:2020C00045F070030220DD749E75F0F0C0E0C0F0122747158115811220DE12223A2274D210
:2020E00075F0F0C0E0C0F012274715811581740290F2D8F090F2D8E075F0007B087C00121F
:202100002B5745F0700302213E800C90F2D8E00490F2D8F01480DD74DB75F0F0C0E0C0F0BB
:2021200090F2D8E075F000C0E0C0F0740275F000122736158115811581158102210B740A62
:2021400075F000C0E0C0F012275A1581158174E175F0F0C0E0C0F0122747158115817400F1
:2021600090F2D9F090F2D9E075F0007B0F7C00122B5E45F0700302221F800C90F2D9E0041D
:2021800090F2D9F01480DD74E575F0F0C0E0C0F090F2D9E075F000C0E0C0F0740275F000BA
:2021A0001227361581158115811581740290F2D8F090F2D8E075F0007B087C00122B574521
:2021C000F0700302221C800C90F2D8E00490F2D8F01480DD90F2D8E090F2DAF090F2DAE015
:2021E00075F0007B047C00122AF990F2DAF074EF75F0F0C0E0C0F090F2DAE090F2D9122B22
:20220000AD4B75F000C0E0C0F0740275F00012273615811581158115810221C802217B22C4
:2022200090F2E6E0122AA97B71122AA0122B4445F070030222390200002290F002E0A3F505
:20224000F0E0C5F0C0E0C0F0122747158115812290F2E6E0122AA97B0D122AA0122B444584
:20226000F0700302227E90F000E0A3F5F0E0C5F0C0E0C0F01227471581158112223A2290C0
:20228000F2E6E0122AA97B64122AA0122B4445F0700302234874F575F0F0C0E0C0F0122709
:2022A0004715811581740E75F0F1C0E0C0F01227471581158179DC7AF2E98AF0C0E0C0F063
:2022C000740A75F000C0E0C0F01227A2158115811581158179DC7AF2E98AF0C0E0C0F01212
:2022E00028031581158190F2E7F0A3C5F0F0C5F0742675F0F1C0E0C0F0740175F0001227DE
:202300003615811581743875F0F1C0E0C0F090F2E7E0A3F5F0E0C5F0C0E0C0F090F2E7E00A
:20232000A3F5F0E0C5F0C0E0C0F090F2E7E0A3F5F0E0C5F0C0E0C0F0740475F0001227362E
:202340007FF8122A8312223A2290F2E6E0122AA97B72122AA0122B4445F070030223A87457
:202360004875F0F1C0E0C0F012274715811581746675F0F1C0E0C0F079007A0289828A8336
:20238000E075F000C0E0C0F079007A0289828A83E075F000C0E0C0F0740375F000122736BB
:2023A0007FFA122A8312223A2290F2E6E0122AA97B69122AA0122B4445F070030224427463
:2023C0007275F0F1C0E0C0F012274715811581749275F0F1C0E0C0F012274715811581746D
:2023E000B375F0F1C0E0C0F01227471581158174D375F0F1C0E0C0F01227471581158174CB
:20240000F375F0F1C0E0C0F012274715811581741375F0F2C0E0C0F0122747158115817429
:202420003375F0F2C0E0C0F012274715811581745375F0F2C0E0C0F01227471581158112EA
:20244000223A2290F2E6E0122AA97B62122AA0122B4445F07003022515747A75F0F2C0E0CE
:20246000C0F012274715811581749975F0F2C0E0C0F01227471581158112260E90F2E9F0FF
:20248000A3C5F0F0C5F074AC75F0F2C0E0C0F012274715811581740090F2D8F090F2D8E0D4
:2024A00075F0007B107C00122B5745F07003022512800C90F2D8E00490F2D8F01480DD7442
:2024C000CA75F0F2C0E0C0F090F2E9E0A3F5F0E0C5F0C0E0C0F090F2E9122BB889828A835B
:2024E000E075F000C0E0C0F0740375F0001227367FFA122A8390F2E9E0A3F5F0E0C5F0124A
:202500002B0A90F2E9F0A3C5F0F0C5F0122B130224B312223A2205810581058105810581D7
:20252000740075F00078FD122A77F608A6F078FD122A77E60886F07B027C00122B2445F0EB
:202540007003022588801678FD122A77E60886F0122B0A18F608A6F0122B1380D178FD121C
:202560002A77E60886F079FA122A7C122A99C001C002122772C0E0C0F012275A1581158119
:20258000D007D000F602254778FD122A77E60886F079FA122A7C122A997400F7740075F060
:2025A0000079FA122A7C122A99E7C39430122AA97B04122AA0122AF9C0E0C0F0740175F00E
:2025C0000079F8122A7C122A99E7C39430D004D0034BC5F04CC5F0122AA97FFB022A92903A
:2025E000F2E6E0122AA97B3F122AA0122B4445F0700302260D90F004E0A3F5F0E0C5F0C009
:20260000E0C0F01227471581158112223A22058105810581058112264D78FB122A77F6082D
:20262000A6F012264D78FD122A77F608A6F0181818E60886F07B087C00122AF90846C5F0E0
:202640000846C5F015811581158115812205810581122772C0E0C0F012283C15811581C094
:20266000E0C0F012275A1581158178FD122A77F6122772C0E0C0F012283C15811581C0E0B0
:20268000C0F012275A1581158178FE122A77F618E6122AA9C0E0C0F01226CE158115817BCC
:2026A000047C00122AF978FD122A77F608E6122AA9C0E0C0F01226CE1581158178FE122A40
:2026C00077F618E60846122AA9158115812278FB122A77E6122AA9C0E0C0F01228B5158148
:2026E000158145F070030226F878FB122A77E6C39430122AA902273578FB122A77E6122A5E
:20270000A97B41122AA0122B3D45F0600CE6122AA97B46122AA0122B2B45F0700302272F8D
:2027200078FB122A77E6C39437122AA9022735740190F2DBF02223F42581F8122B95122916
:2027400009122B9502275178FB122A778682088683E0602D122760A380F778FB122A77E6B9
:202760003099FDC299F599B40A17740D80F2E430980C3098FDC298E599B40D02740A75F0E7
:20278000002278FB122A77E63099FDC299F5992274FFF5F030980A3098FDC298E59975F00E
:2027A000002278FC122A778604188603188683188682E4FDFE122772B408028003B47F273F
:2027C000ED4E60F11DBDFF011E7408122760742012276074081227608583F0E582122B136F
:2027E00085F083F58280CE122760F024F3600EA30DBD00010EED8EF0122B2470B8E4F0EDDD
:202800008EF02278FB122A778682088683E4FBFCFFE0A3B42D030FE0A3C39430B40A005071
:2028200012FA740A75F000122AB22AFBE5F03400FC80E4EB8CF0DF03022B1A2278FB122ACC
:2028400077E6C0E008E6C0E012288913D0F0D0E0500224E02278FB122A77E6C0E008E6C0D5
:20286000E012288E13D0F0D0E050E9242022D005D0061228B56009C006C00522D005D00633
:2028800012288E70F2C006C00590617A802A90415A802590217E802090007F801BD005D080
:2028A000069041461228B870CE9061661228B870C6C006C00590303978FB122A77E6B58384
:2028C00000400DB5820808E67006F5F0042240F6E4F5F02278FB122A77E690001FB47FDE10
:2028E00080E4D003D00412286EC004C00370E190207E80C478FB122A77E6C3940960C71434
:2029000060C4C3941660BF80C7122A50868208868308E4FEFFE07006122A50E4F022B42581
:2029200051A3E0B42D05430780A3E0B4300343074024D0B40A00500BCE75F00AA42EFEA362
:20294000E080EEE0B46413E60886F030F708430720122B1AA6F018F68003B4750543070A21
:202960008021B478054307108019B46F104307088011122A50F0A3122A50A38095B46262A1
:202980004307027A00C004C005C006C007AB0753031F7C00E60886F0122AC6A6F018F6EDC1
:2029A000D007D006D005D0042430B43A0040022407C0E00AE645F070CC122A50A902EF30BB
:2029C000E505742DF0A30A122A59D0E0F0A3D9FA0808EF30E7A1EAC39E509C7420F0A30A05
:2029E00080F4B4630DAA01122A50122A59E6F0A380DEB47331C082C08386820886837A002C
:202A0000E06004A30A80F98683188682122A50122A59122A50E0A3122A506004F0A380F2FE
:202A2000D005D00480AAB4691B86017A00E76004090A80F9122A50122A598601E76091F043
:202A400009A380F8F97A01122A50122A59E9809ECDC583CDCCC582CC22EE601A8FF020F7D5
:202A600015C002EAC39E500C742030F6027430F0A30A80EFD00222C82581C822C92581C9E8
:202A80007A0022D083D082CF2581F581CFC082C08322CF2581F581CF2229F9E5F03AFA226B
:202AA0007C00CB30E7011CCB2275F00030E70215F022FEEBA4FD8EF0ECA4FCEB8EF0A4C5A3
:202AC000F02C2DC5F022C002C001AAF0F97E007D007F11C3E933F9EA33FADF08F5F0E9D0C1
:202AE00001D00222ED33FDEE33FEC3ED9BF5F0EE9C40E0ADF0FED380DBBB000122C333C569
:202B0000F033C5F0DBF722122B0A04700205F022122B1314B4FF0215F022122B13F4C5F0DC
:202B2000F4C5F022122B774029801E122B7740227017801E122B7740107017800C122B7709
:202B400050108005122B8B6009E4F5F022122B8B60F7E4F5F00422122B8B40F680EB122BC0
:202B60008B40EF70E480EB122B8B40DD70E480D9122B8B50DD80D2C39BC5F09C20E7072026
:202B8000D207C345F02220D2F9D322C5F0C39C7003E5F09B2290F2EBE0A360F8E0FFA3E09F
:202BA000A3CF2582F582EF3583F58380EBFBE0CB22FCE0FBA3E0CC22FAE0F9A3E0CA2206A3
:202BC000F03DF042F00A0A38303531534243206E657720636F6D6D616E6473202870726581
:202BE0007373203F20666F722068656C70206F72207120746F207175697429000A0A3E3E2F
:202C0000000A0A48656C70204D656E750A41204153434949205461626C650A44204465630C
:202C2000324865780A522052656164204750494F320A5120517569740A4920692F6F2061AB
:202C40006464726573730A422042696E61727920696D6167650A3F2068656C70007072699E
:202C60006E7461626C6520415343494920636F64657328686578292C20652E672E20415369
:202C8000434949206F6620274127206973203431000A0A2020204D534200202020256400FB
:202CA0004C5342000A202025317820202000202020256300446563696D616C20746F2048B9
:202CC000657820636F6E766572746572000A0A456E74657220646563696D616C206E756DAE
:202CE0006265723D00446563202D3E20486578202D3E2042696E000A2564202D3E202578E3
:202D0000202D3E2025620052656164204750494F322028382D62697420696E7075742070B8
:202D20006F727429000A0A25303278202530386200692F6F206465636F64657220616464AD
:202D400072657373206D61646520627920504C44000A0A4C4344202020636F6D6D616E64DE
:202D60002077726974652020202020307830303030000A4C43442020206461746120777220
:202D80006974652020202020202020307830303031000A4C4344202020636F6D6D616E646C
:202DA0002072656164202020202020307830303032000A4C4344202020646174612072655F
:202DC0006164202020202020202020307830303033000A4750494F3120382D626974206FE6
:202DE000757470757420706F727420307830313030000A4750494F3220382D62697420696B
:202E00006E7075742020706F727420307830323030000A657870616E73696F6E20692F6F56
:202E200020737061636520202020203078303330302D3078303746460073656520686F77E8
:202E4000207265616C2070726F6772616D206C6F6F6B206C696B65000A0A656E74657220AA
:202E600061646472657373203D20000A0A4131352E2E2E2E2E2E2E2E2E2E2E2E4130204437
:172E8000372E2E2E2E2E4430000A2025303136622020253038620033
:10500000A5E5E0A5FD46000000000000000000004E
:10501000000000000000000000000000FFFFFFFF94
:10502000383035312043616D656C20464F5254480D
:0250300020005E
:10504000900200E030E1012290507FE5838582F0FC
:1050500090800CF0A3E5F0F090800B7402F0025009
:10506000B4C0D0C0E0C082C083E5742401F574856B
:105070003F8385C782E0D083D082D0E0D0D032C0D9
:10508000D0C0E0758CDC758A00E5702401F570E411
:105090003571F571E43572F572E43573F573D0E06E
:1050A000D0D03275A800758700758920758DFDD226
:1050B0008E7598527508FE8508A078FF7581087571
:1050C0007000757100757200757300758921758C9B
:1050D000DC758A00757400D28CD28875A88302684A
:1050E000F700000004454D49543099FDC29985826E
:1050F000994103E45000034B45593098FDC298187C
:10510000E583F218E582F285998275830022F650D4
:1051100000044B45593F18E583F218E582F2E59803
:105120001381C1115100044558495415811581223C
:10513000265100034C495418E583F218E582F2D059
:1051400083D082E493A3FAE493A3C082C083F5835F
:105150008A82223351000745584543555445C08241
:10516000C0834103565100085641524941424C45C3
:1051700012654212582F02609B67510008434F4E40
:105180005354414E5412654212582F1253F8126074
:10519000E11260ED12658418E583F218E582F2D021
:1051A00083D08261447C51000455534552318512AD
:1051B000658431E3D083D08271442508F5832231A0
:1051C000E3D083D0822218E583F218E582F2D0057D
:1051D000D004D083D082C004C0056144A85100032C
:1051E00044555018E583F218E582F222DF5100049D
:1051F0003F445550E583458270E922EF5100044455
:10520000524F50E2F58208E2F5830822FE51000475
:1052100053574150E2FA08E2FBE583F218E582F2C7
:105220008B838A82220F5200044F564552E2FA08BD
:10523000E2FB181880E328520003524F54E2FC08A6
:10524000E2FD08E2FA08E2FBEDF218ECF21880C980
:10525000395200023E52D003D002C082C083C00245
:10526000C003809F53520002523E18E583F218E5B6
:1052700082F2D003D002D083D082C002C003226762
:10528000520002524018E583F218E582F2A9811912
:10529000198783198782228252000353504018E5F0
:1052A00083F218E582F28508838882229A520003ED
:1052B000535021A8824103AF52000352504018E5D9
:1052C00083F218E582F275830085818222BA52004A
:1052D00003525021D003D002858281C002C0034115
:1052E00003D05200034E495051144103E4520004CC
:1052F0005455434B5114412DEF52000121E208F067
:10530000A3E208F04103FB5200024321E208F00847
:1053100041030953000140E0FAA3E08A82F58322A9
:10532000155300024340E0F58275830022235300A9
:1053300002492180C83053000349432180CE3853AD
:1053400000024940E493FA7401938A82F583224172
:10535000530002494340E493F5827583002252537F
:1053600000012BE2082582F582E2083583F58322CD
:10537000615300024D2BE2FA08E2FB08E22582F2BB
:1053800008E23583F218E43AF582E43BF5832273B0
:105390005300012DE208C39582F582E2089583F55A
:1053A000832292530003414E44E2085582F582E283
:1053B000085583F58322A55300024F52E208458227
:1053C000F582E2084583F58322B9530003584F5212
:1053D000E2086582F582E2086583F58322CC5300FA
:1053E00006494E564552546382FF6383FF22E053C1
:1053F00000064E45474154456382FF6383FFA32265
:10540000F1530002312BA32203540002312DE58217
:10541000700215831582220B5400023E3CE5828502
:105420008382F583221A540002322AE5822582F50E
:1054300082E58333F5832228540002322FE583333B
:10544000E58313F583E58213F582223A5400064C76
:105450005348494654AC82E2F58208E2F583080CD1
:10546000800BE5822582F582E58333F583DCF32228
:105470004E540006525348494654AC82E2F5820825
:10548000E2F583080C800BC3E58313F583E58213F3
:10549000F582DCF322735400022B21E208FAE02AA1
:1054A000F0A3E208FAE03AF04103985400023C3ECF
:1054B00091D88006AD540002303DE5834582C39407
:1054C0000195E0F583F58222B7540002303CE58374
:1054D0003380EECB5400013D719480E0D65400013E
:1054E0003C719430D201F43380D7DF5400013E5137
:1054F0001480EEED540002553C719480C4F65400C3
:1055000002553E511480F2005500073F4252414E71
:105510004348E2FA08E208C58345828A82220A5596
:105520000006284C4F4F5029EE2401FEEF3400FFB7
:1055300020D220E42221550007282B4C4F4F502920
:10554000EE2582FEEF3583FFE2F58208E2F583085F
:1055500030D2E0E4F4223855000428444F29D00327
:10556000D002C006C007E208F42401FCE208F434CB
:1055700080FDC004C005EC2582FEED3583FFC0022E
:10558000C0034103595500014918E583F218E5822B
:10559000F2A981191919C3EE97F58209EF97F583DE
:1055A00022875500014A18E583F218E582F2A981A5
:1055B0001919191987031987021987F019C3EA976E
:1055C000F582EB95F0F58322A4550006554E4C4F1D
:1055D0004F50D003D00215811581D007D006C002EC
:1055E000C00322CB550003554D2AE2F908E9858214
:1055F000F0A4FAABF0E98583F0A42BFBE435F0FCD2
:10560000E28582F0A42BFBEC35F0FCE43400FDE2F3
:105610008583F0A42CFCED35F0F5838C82EBF21839
:10562000EAF222E6550006554D2F4D4F44E2FB08A5
:10563000E2FA08E2FD08E2FC7911C38029EB33FBB2
:10564000EA33FA500CC3EB9582FBEA9583FAC380E8
:1056500014C3EB9582FBEA9583FA5009EB2582FB94
:10566000EA3583FAD3B3ED33FDEC33FCD9CF8D8229
:105670008C83EAF218EBF2222656000446494C4C81
:10568000AC82E2FA08E2FB08E2F58208E2F5830860
:10569000EC0B0A8002F0A3DAFCDBFA41037B560034
:1056A00004492D3E4431F4B112601A512D716351F9
:1056B00014B15E31E37156B189710C9106B1286065
:1056C000F2B1D231E351034103A0560004442D3E10
:1056D000498009CC560005434D4F564531F4B1126F
:1056E000601A512D71635114B15E31E37126B18995
:1056F000710C9106B12860F2B1D231E3510341033C
:10570000D6560006434D4F56453E31F4B11260283F
:10571000910E513D512D7163513D513D512D71639C
:10572000B15E31E37126B189710C910E3137FFFF03
:10573000B14060EEB1D231E351034103035700049D
:10574000534B4950AC82E2FA08E2FB08E2F58208CA
:10575000E2F5830B0A8005E06C7005A3DAF9DBF74C
:10576000E583F218E582F21A1B8B838A82A3223F1B
:105770005700045343414EAC82E2FA08E2FB08E2D0
:10578000F58208E2F5830B0A8005E06C6005A3DA78
:10579000F9DBF7E583F218E582F21A1B8B838A8224
:1057A000A322725700024E3DC007C006AA82AB83F7
:1057B000E2FC08E2FD08E2FE08E2FF080B0A803A7C
:1057C0008D838C82E493C39461400A941A5006E45A
:1057D0009364208002E493F9A3AD83AC828F838E1F
:1057E00082E0C394614009941A5005E0642080016E
:1057F000E0A3AF83AE82C399700ADAC4DBC28B83A5
:105800008B82800895E0F5834401F582D006D007AD
:1058100022A5570005414C49474E22145800074124
:105820004C49474E4544221E58000443454C4C12F7
:10583000519702002A58000543454C4C2BA3A32244
:105840003758000543454C4C5302542B4358000530
:10585000434841522BA3224F58000543484152531D
:10586000225A5800053E424F4459A3A3A302534471
:1058700064580008434F4D50494C452C1251371283
:105880000012610012541D0260ED735800032143A1
:1058900046125137120012522D12533C1254061266
:1058A000521412541D1252140253338D5800032CFB
:1058B000434680C8AE58000621434F4C4F4E12510C
:1058C00037FBFF0260E1B75800052C4558495412D8
:1058D00051372200026100C95800072C4252414E44
:1058E00043481251F4125512600B12587C12513772
:1058F00060000261001251378000026100DA580036
:10590000052C444553541260D1125406125394028C
:1059100061000059000521444553541252F41254B9
:105920000612539412521402533C155900072C5579
:105930004E4C4F4F50125137D25502587C2D5900C2
:1059400002424C12519720004059000754494253DB
:10595000495A451251977E004B590003544942124F
:1059600051B280FF5B59000255301251B2000067FE
:105970005900033E494E1251B202007259000442CE
:105980004153451251B204007E590005535441540D
:10599000451251B206008B59000244501251B20810
:1059A000009959000727534F555243451251B20AE7
:1059B00000A45900064C41544553541251B20E00F4
:1059C000B459000248501251B21000C35900024CA1
:1059D000501251B21200CE5900034944501251B234
:1059E0001400D959000253301251B2FF00E559009A
:1059F000035041441251B22801F05900024C3012B8
:105A000051B28001FC59000252301251977F0007B9
:105A10005A000555494E49541251BF00000000106C
:105A200000000000D00000000069700000000000CD
:105A300090125A000523494E4954125197160034CA
:105A40005A0003533E441251E30254CE425A000717
:105A50003F4E45474154451254CE12551260031231
:105A600053F8224F5A00034142531251E380E86633
:105A70005A0007444E45474154451252141253E709
:105A80001252141253E71251370100025376725A20
:105A900000083F444E45474154451254CE1255121A
:105AA0006002517A22915A0004444142531251E358
:105AB00080E8A85A00024D2A91221253D012525661
:105AC000125214516A125214516A1255EA12526A51
:105AD00080C8B55A0006534D2F52454D912212539E
:105AE000D012525612522D125256516A125256511B
:105AF000AD12526A12562D12521412526A51571296
:105B0000521412526A4157D55A0006464D2F4D4F36
:105B1000441251E312525691221253D0125256128D
:105B2000525651AD125285516A12562D125214120C
:105B3000526A515712521412526A1254CE1255120E
:105B4000601A1253F812522D125512600F1252851C
:105B500012523D12539412521412540E12526A12DF
:105B60005203220A5B00012A51B8025203665B000D
:105B7000042F4D4F44125256514612526A61117011
:105B80005B00012F71750252E8825B00034D4F44A8
:105B900071750252038C5B00052A2F4D4F4412523F
:105BA0005651B812526A6111985B00022A2F719EF9
:105BB0000252E8AB5B00034D415891221254E112AE
:105BC00055126003125214025203B65B00034D4992
:105BD0004E91221254EF12551260031252140252C7
:105BE00003CD5B000232401251E312583D125317AD
:105BF000125214025317E45B0002322112521412A3
:105C0000522D1252FD12583D0252FDF95B00053231
:105C100044524F501252030252030E5C00043244AD
:105C2000555012522D02522D1D5C00053253574122
:105C30005012523D12525612523D12526A222B5CA1
:105C40000005324F564552125256125256912212A8
:105C5000526A12526A8131415C0005434F554E54DD
:105C60001251E31258551252140253265A5C000284
:105C700043521251370D001250E91251370A0002F7
:105C800050E96F5C0005535041434512594302509F
:105C9000E9855C00065350414345531251E31255C8
:105CA000126007918B12540E80F1025203945C0033
:105CB00004554D494E91221255031255126003129C
:105CC0005214025203B05C0004554D415891221207
:105CD00054F91255126003125214025203C85C00A8
:105CE0000555434153451251E31252561251376143
:105CF000001251377A00126808125512600D1252C4
:105D00006A12513720001253D0800312526A22E0E7
:105D10005C00075541434345505412522D125363C2
:105D200012540E12522D1250FA125CE61251E31266
:105D300051370D001254B012551260391251E3124E
:105D400050E91251E312513708001254D81255127B
:105D5000601312520312540E12525612522D125246
:105D60006A91CD800E12522D12530C12540612520B
:105D70002D91B580B11252031252E81252140253FF
:105D800094125D000641434345505412522D125364
:105D90006312540E12522D1250FA1251E31251375F
:105DA0000D001254B012551260391251E31250E92D
:105DB0001251E312513708001254D81255126013D1
:105DC00012520312540E12525612522D12526A914E
:105DD000CD800E12522D12530C12540612522D91D8
:105DE000B580B41252031252E81252140253948432
:105DF0005D0004545950451251F4125512601F129F
:105E0000522D12536312521412555E1255891253B9
:105E1000261250E912552860F21255D28003125210
:105E20000322F25D0005284953222912526AD1D07B
:105E3000912212536312525622255E0004285322E7
:105E40002912528512534412526A12583D1251E3DC
:105E5000125356125855912212536312525612522F
:105E60005612522D12526A1256A581603C5E0103F1
:105E70004953221251372B5E12587C12513722009F
:105E8000125F191253561254060260E16F5E01024E
:105E90005322125137415E12587C12608C1260ED11
:105EA0001251372200F1191253561254061251E3BF
:105EB00012609B0260E18F5E01022E22D1731251AB
:105EC00037E55E02587CB95E000649434F554E5493
:105ED0001251E3125855125214025356C95E00056E
:105EE00049545950451251F4125512601F12522D47
:105EF00012536312521412555E12558912535612E0
:105F000050E912552860F21255D280031252032232
:105F1000DF5E000549574F524412615D1260D11295
:105F200052F412522D1253261258550256D1135FB5
:105F3000000655442F4D4F4412525612513700005F
:105F400012528512562D12523D12523D12526A12B1
:105F5000562D02523D315F000355442A1251E3127F
:105F600052561255EA12520312521412526A125524
:105F7000EA12523D025363585F0004484F4C4412EA
:105F80005137FFFF31C612549B31C61253170253CB
:105F90000C7A5F00023C2331F431C60252FD945F5B
:105FA00000063E44494749541251E3125137090053
:105FB0001254EF12513707001253A91253631251B2
:105FC000373000025363A15F00012331831253175E
:105FD000F13812523DF1A880A6C95F00022353F1A7
:105FE000CB91221253BC1254BA12551260F122DC2A
:105FF0005F0002233E911431C612531731F412523E
:106000002D025394F25F00045349474E1254CE12AE
:10601000551260081251372D00125F7F2207600071
:1060200002552E125F971251370000125FDF125F88
:10603000F5125DF7025C8B206000012E125F971253
:1060400051E3125A6A1251370000125FDF12523DBB
:1060500012600C125FF5125DF7025C8B3A6000076C
:10606000444543494D414C1251370A0012598302AD
:1060700052FD5F6000034845581251371000125915
:10608000830252FD756000044845524512599C0236
:10609000531787600005414C4C4F5412599C0254D1
:1060A0009B956000012C12608C1252FD1251370238
:1060B0000002609BA4600002432C12608C12530CFF
:1060C000125137010002609BB760000549484552F4
:1060D000451259DD025317CB60000649414C4C4F25
:1060E000541259DD02549BDA600002492C11D1127E
:1060F0005333125137020080E8EA60000349432C11
:106100001260D112533C125137010080D4FC600060
:1061100006534F555243451259AC025BE7106100DC
:10612000072F535452494E4712523D12522D1253CB
:106130006312523D12523D025394206100083E43C7
:106140004F554E544544125C2212530C12585512AE
:1061500052140256DC3D610004574F52441251E381
:106160001261171259761253171261281251E31255
:10617000525612523D12574412522D12525612527A
:106180003D1257771251E3125512600312540E124A
:10619000526A12526A12523D125394125976125494
:1061A0009B1252F412539412608C12614612608C4E
:1061B00012594312522D125C6012536302530C5851
:1061C0006100074E46413E4C4641125137030002E2
:1061D0005394C26100074E46413E434641125ED091
:1061E0001251377F001253A9025363D5610006494B
:1061F0004D4D45443F12540E025356EE6100044685
:10620000494E441259BB125317125C2212522D12DE
:1062100053261258551257A81251E3125512600C0A
:106220001252031261CA1253441251E31254BA12A9
:10623000551260D51251E312551260181252E8122D
:1062400051E331DD12521431F51254BA12513701B3
:10625000001253BC22FE6101074C49544552414C87
:10626000125991125317125512600B1251373751B0
:1062700012587C1260ED2258620006444947495486
:106280003F125CE61251E312513739001254EF12FB
:10629000513700011253A91253631251E3125137BF
:1062A00040011254EF12513707011253A9125394AF
:1062B00012513730001253941251E3125983125382
:1062C000170254F97A6200053F5349474E12522D86
:1062D0001253261251372C001253941251E3125AC2
:1062E0006A12513701001254D81253A91251E31205
:1062F00055126011125406125256125137010012F3
:10630000612812526A22C76200073E4E554D42452F
:10631000521251E3125512603612522D12532612A8
:1063200062811254BA12551260030252031252567D
:10633000125C31125983125317125F5C12526A12A7
:106340005376125C31125137010012612880C2224B
:10635000096300073F4E554D4245521251E3125119
:106360003700001251E312523D125C601262CD12EE
:106370005256126311125512601012526A125C14B6
:10638000125C1412513700008016125C141252E88D
:1063900012526A12551260031253F8125137FFFF5E
:1063A0002253630009494E544552505245541259E4
:1063B000AC125BFC12513700001259761252FD12DA
:1063C000594312615D1251E3125326125512604B6C
:1063D0001262031251F4125512601E125406125921
:1063E000911253171254BA1253BC1255126005126F
:1063F000515E800312587C8020715B12551260053B
:106400001262608014125C60125DF71251373F0017
:106410001250E9125C721264AE80A4025203A463AB
:1064200000084556414C554154451259AC125BE7A2
:106430001252561252561259761253171252567160
:10644000AE12526A1259761252FD12526A12526AF2
:106450001259AC025BFC2164000451554954125995
:10646000FF1259D11252FD125A0A1252D412513748
:1064700000001259911252FD12595F1251E3125944
:1064800053125D8B125C8B71AE125991125317121D
:1064900054BA1255126009125E2B026F6B125EE540
:1064A000125C7280D35964000541424F5254125914
:1064B000E81252B380A8A86400063F41424F5254EC
:1064C00012523D1255126005125EE580E1025C1425
:1064D000B964010641424F525422125E7312513781
:1064E000C06402587CD36400012712594312615DD5
:1064F0001262031254BA125E2B013F80C3E864009B
:10650000044348415212594312615D12540602532A
:1065100026006501065B434841525DB105125137C3
:10652000375112587C0260ED146501012812513771
:10653000290012615D0252032B650006435245415A
:1065400054451259BB1253171260ED125137000017
:106550001261001260D11259BB1252FD125943123E
:106560005F191253561254061260E11251379751B7
:106570001258B212608C0260ED3B65000728444F50
:1065800045533E2912526A1259BB12531731DD028C
:1065900058917C650105444F45533E12513784653F
:1065A00012587C125137C6510258B29565010752F4
:1065B0004543555253451259BB12531731DD02580A
:1065C0007CAE6501015B12513700001259910252F5
:1065D000FDC46500015D125137FFFF12599102524F
:1065E000FDD4650004484944451259BB12531712A3
:1065F00051E312535612513780001253BC125214F9
:1066000002533CE465000652455645414C1259BBC5
:106610001253171251E31253561251377F0012537F
:10662000A912521402533C06660009494D4D4544D7
:106630004941544512513701001259BB12531712E8
:10664000540E02533C2A6600013AB142B1E9B1D678
:106650000258BE486601013BD10D1258CFA1C65663
:106660006601035B275D91EA125137375112587C5E
:106670000260ED62660108504F5354504F4E451270
:10668000594312615D1262031251E31254BA125E51
:106690002B013F1264C01254CE12551260151251D4
:1066A00037375112587C1260ED1251377C5812580E
:1066B0007C800312587C22766601024946125137CB
:1066C00012551258E21260D11251E3025906BA660D
:1066D00001045448454E1260D112521402591BD184
:1066E000660104454C534512513700001258E2121E
:1066F00060D11251E312590612521480D9E2660198
:1067000005424547494E0260D100670105554E5488
:10671000494C12513712551258E20259060C6701C2
:1067200005414741494E12513700001258E20259C3
:1067300006206701055748494C45D1BD0252143423
:10674000670106524550454154F126808942670051
:10675000023E4C12582F1259D112549B1259D11289
:1067600053170252FD506700024C3E1259D112538A
:106770001712531712582F1253F81259D102549B63
:1067800068670102444F1251375E5512587C1260FF
:10679000D11251370000E15383670007454E444C46
:1067A0004F4F501258E2125906125935F16B1251DF
:1067B000F41255126004D1D680F2229B6701044C7A
:1067C0004F4F50125137285580D9BE6701052B4CC9
:1067D0004F4F50125137405580C9CD6701054C4588
:1067E000415645125137D25512587C12513700008C
:1067F0001258E21260D11251E3125906E153DD67DB
:10680000000657495448494E12522D1253941252C1
:106810005612539412526A0254F9016800044D4F03
:106820005645125256125C221252141251E3125261
:1068300085125363126808125512600812526A12C8
:10684000570A800612526A1256DC221D680005445F
:106850004550544812529E1259E812521412539441
:1068600002543D4E68000C454E5649524F4E4D4520
:106870004E543F125C141251370000226668000526
:10688000574F5244531259BB1253171251E3125E21
:10689000D01251377F001253A9125EE5125C8B12A1
:1068A00061CA1253441251E31254BA12551260DBFA
:1068B0000252037F6800022E5312529E1259E812B0
:1068C0005394125512602712529E1259E8125137F2
:1068D000020012539412555E12558912531712601A
:1068E00023125137FEFF12554060ED1255D222B6E9
:1068F000680004434F4C44125A1812596A125A3A0B
:106900001256A5125E2B22383035312043616D6559
:106910006C466F7274682076312E36203237204DE7
:10692000617220323030300D0A125EE51259E812E1
:1069300052B31259FF1259D11252FD125A0A125271
:10694000D412513700001259911252FD126E1802E2
:1069500064AEE583858283F5822253820F758300BE
:10696000225382F0E58203030303F582758300223C
:10697000E582C3940A40022407243AF5821250E9C2
:10698000221251E312696112697012695A12697018
:10699000221251E31253261269811251372000123C
:1069A00050E9125406221251E3126CC2126981128C
:1069B000513720001250E9125406221251E31253AB
:1069C0004412698112513720001250E912540622F4
:1069D0001251E312695212698112698112513720F2
:1069E000001250E922F268000444554D501251370C
:1069F000000012555E125C721251E31269D0125CF3
:106A00008B126991126991126991126991126991BF
:106A10001269911269911269911269911269911228
:106A200069911269911269911269911269911269C1
:106A300091125137100012554060BA1255D21252BD
:106A40000322E86900054944554D501251370000B2
:106A500012555E125C721251E31269D0125C8B12F5
:106A600069A61269A61269A61269A61269A6126918
:106A7000A61269A61269A61269A61269A61269A6CB
:106A80001269A61269A61269A61269A61269A6124F
:106A90005137100012554060BA1255D212520322DB
:106AA000456A00054344554D5012513700001255B8
:106AB0005E125C721251E31269D0125C8B1269BBD8
:106AC0001269BB1269BB1269BB1269BB1269BB12A6
:106AD00069BB1269BB1269BB1269BB1269BB12693F
:106AE000BB1269BB1269BB1269BB1269BB12513779
:106AF000100012554060BA1255D212520322A36AF6
:106B00000003215031858290025203016B00034043
:106B100050311251E3859082758300220E6B000381
:106B20002150348582C00252031F6B000340503451
:106B30001251E385C082758300222C6B000521541D
:106B4000434F4E8582880252033D6B0005405443FB
:106B50004F4E1251E3858882758300224C6B0006EC
:106B6000405331434F4E1251E385D8827583002242
:106B70005F6B00064053315354411251E385D98273
:106B800075830022736B0006405331414452125109
:106B9000E385DB8275830022876B00062153314138
:106BA00044528582DB0252039B6B00074932434902
:106BB0004E495412380022AB6B000A40493243530D
:106BC0005441545553123806C0E01251E3D0E0F559
:106BD0008275830022BA6B0006493243434D44124A
:106BE0003803F58275830022D86B00093240434C8C
:106BF0004B5449434B1251E3857183857082125186
:106C0000E385738385728222EB6B000344303C087A
:106C100008E5833395E0F583F582220B6C0002448E
:106C20002D1251E3E82406F9E82402F8E2FAE3C35E
:106C30009AF30809E2FAE39AF3181818191919E2F5
:106C4000FAE39AF30809E2FAE39AF3080808E2F58E
:106C50008208E2F58308221E6C0002442E125214B0
:106C600012522D125AAD125F97125FDF12523D126F
:106C7000600C125FF5125DF7025C8B5A6C000355D5
:106C8000442E125F97125FDF125FF5125DF7025C10
:106C90008B7E6C000544454C4159125256126BF5DF
:106CA00012526A125376125C22126BF5126C211288
:106CB0006C0F12551260EF125C1422946C000349A1
:106CC0004440E582F9E7F58275830022BE6C00033B
:106CD000494421E582F9E2F70808025203CF6C002B
:106CE00004412F4421E5C55407F5C5E5825407D278
:106CF000E3F5C5025203E06C0004412F4440E5C5B2
:106D000030E4FB1251E385C683E5C554C0F5821219
:106D100051E375820675830012547A22F96C0006DD
:106D20004144434F4E401251E385C5827583002292
:106D30001F6D00064144434F4E218582C502520318
:106D4000336D000541444348401251E385C68275C6
:106D5000830022436D000550574D50218582FE026D
:106D60005203566D000550574D50401251E385FEB9
:106D70008275830022656D000550574D3021858254
:106D8000FC025203786D000550574D30401251E31C
:106D900085FC8275830022876D000550574D312197
:106DA0008582FD0252039A6D000550574D31401205
:106DB00051E385FD8275830022A96D000753455478
:106DC00042414E4BE582134004C2908002D29013A0
:106DD0004004C2918002D291134004C2928002D238
:106DE00092025203BC6D00094D53454344454C414A
:106DF00059AB82AC83BB0006BC000302520379E5A9
:106E0000A3D9FD1BBBFFEE1C80F4025203E76D000B
:106E100007465448424F4F541251E3758300758220
:106E200007126DC41251E375830075820012532658
:106E30001251E37583007582281254D812551260DE
:106E4000731251E37583207582001251E37583003C
:106E500075820012555E1255891253261251E37540
:106E600083007582FF1254D8125512603F125E2BB8
:106E7000154576616C75617465204550524F4D2003
:106E8000757020746F3A125EE512558912603C12DB
:106E900051E375830075820012558912642A125ECF
:106EA0002B046F6B0D0A125EE50264AE125528606A
:106EB000A51255D222106E0004545255451251E3CA
:106EC00090FFFF22B86E000546414C53451251E336
:106ED00090000022C76E0008534156455F494D4758
:106EE00012525612608C1252851252FD1260D1124B
:106EF00052851251E39000021253631252FD12594F
:106F0000BB1253171252851251E3900004125363BF
:106F10001252FD1270271252851251E39000061290
:106F200053631252FD1251E390D000125285125158
:106F3000E390000812536312608C1251E390D0006A
:106F40001253941268B91256DC1251E39090001259
:106F5000526A1251E390000812536312608C12516E
:106F6000E390D0001253941253631260D11251E394
:106F70009090001253941268B91256DC22D76E001A
:106F8000084C4F41445F494D4712525612528512E8
:106F9000531712599C1252FD1252851251E3900060
:106FA000021253631253171259DD1252FD12528509
:106FB0001251E39000041253631253171259BB127B
:106FC00052FD1252851251E3900008125363125180
:106FD000E390D00012608C1251E390D000125394D1
:106FE0001268B91256DC12526A1251E3900008126C
:106FF000536312608C1251E390D0001253941253D9
:10700000631251E39090001260D11251E39090000E
:107010001253941268B91256DC22806F00094C4159
:10702000535449574F52441251E3907069221D70D6
:107030000006535749544348AA83AB8285088315F9
:10704000837582008801E581F0A3F8E6F0A3D8FB00
:107050008A838B82E0A3F581F8E0A3F6D8FBA80130
:107060008508A002520331700008494E495454412A
:10707000534B740AF0A3E208FAE208F0A3EAF0A383
:10708000E58304F0A3A3A3A3A3A3A374FDF002527A
:0170900003FC
:00000001FF
